:1000000019C032C031C030C02FC02EC02DC02CC08E
:100010002BC02AC029C028C027C026C025C024C0A4
:1000200023C022C044C17DC11FC01EC01DC01CC052
:100030001BC01AC011241FBECFEFD2E0DEBFCDBF60
:1000400011E0A0E0B1E0E6E8F8E002C005900D9212
:10005000A432B107D9F711E0A4E2B1E001C01D92CA
:10006000A93AB107E1F701C0CBCFCBEDD2E0DEBFBB
:10007000CDBFCFD08CE080D1789480EF8BB98AB996
:1000800015B814B880E091E09F938F93B8D38BE0BC
:1000900091E09F938F93B3D30F900F900F900F9099
:1000A000BB245B2CAB2C87E191E09F938F93A7D36C
:1000B000EE24FF240F900F903701470181E090E07C
:1000C0000E2C02C0880F991F0A94E2F784B98CE1C4
:1000D00091E09F938F9393D3CC24DD240F900F90C6
:1000E00084010E0D1F1D0C0D1D1D1E010894211CE9
:1000F000311C020D131D8C2D9ED0F8018083992791
:100100009F938F938FE191E09F938F9378D3F80122
:1001100080810F900F900F900F908B3038F5EC147A
:10012000FD0451F481E090E00E2C02C0880F991F6D
:100130000A94E2F7582A1AC085E090E08C199D09CC
:10014000E816F90651F481E090E00E2C02C0880F09
:10015000991F0A94E2F7B82A09C081E090E00E2CBA
:1001600002C0880F991F0A94E2F7A82AF301EE0D46
:10017000FF1DEC0DFD1DE20DF31D80818B50833FB3
:1001800048F481E090E00E2C02C0880F991F0A9479
:10019000E2F7A82A0894C11CD11CF6E0CF16D104BE
:1001A0000CF49ECF0894E11CF11C85E090E0880ED1
:1001B000991E680E791E8E159F050CF07FCF8FEF6C
:1001C000EFE35E1631F4BB2069F4AA2059F48FEEF8
:1001D0001EC0552039F4FFE3BF1621F4AA2011F404
:1001E0008FED15C0A1108F7B9FE3591621F4BB2022
:1001F00021F08F7B02C0552021F0EFE3BE1609F4F9
:100200008F7BFEE3F51518F0FB1508F08F778BB99F
:1002100047CF809164008E7F8093640080E4809358
:100220007C0087E980937A0010927B008FE38093B3
:100230007E0008950895863018F080E090E00895DB
:10024000805A80937C0080917A00806480937A0049
:1002500080917A0086FDFCCF8091790099270895DE
:1002600008958BB199279695879596958795809552
:1002700090958170907008959091A6018091A7014A
:10028000981730F09091A6018091A701981B06C0A5
:100290009091A6018091A701981B905C953110F078
:1002A0005A9A0895903208F45A98089508951F9222
:1002B0000F920FB60F9211242F933F934F935F939A
:1002C0006F937F938F939F93AF93BF93EF93FF931E
:1002D0009091C0002091C6009871E091A601EF5F57
:1002E000EF738091A701E81711F492E006C0E09344
:1002F000A601FF27EC59FE4F20839093A801BCDF95
:10030000FF91EF91BF91AF919F918F917F916F91ED
:100310005F914F913F912F910F900FBE0F901F90C3
:1003200018951F920F920FB60F9211248F939F93DF
:10033000EF93FF939091A4018091A501981771F01C
:100340008091A5018F5F8F738093A501E82FFF2710
:10035000EC5DFE4F80818093C60005C08091C10096
:100360008F7D8093C100FF91EF919F918F910F90AE
:100370000FBE0F901F901895982F1092A401109205
:10038000A5011092A6011092A70188E98093C100EF
:100390009093C4005A98529A08951F939091A60181
:1003A0008091A701981719F480E091E013C0809123
:1003B000A7018F5F8F738093A701E82FFF27EC5968
:1003C000FE4F108159DF8091A8019927982F882727
:1003D000810F911D1F91089520E030E09091A601BA
:1003E0008091A701981711F021E030E0C90108952C
:1003F0001F939091A6018091A7019817D1F31091B6
:10040000A7011F5F1F731093A70136DFE12FFF279E
:10041000EC59FE4F808199271F910895282F9091C4
:10042000A4019F5F9F738091A5019817E1F3E92FC5
:10043000FF27EC5DFE4F20839093A4018091C100C3
:1004400080628093C1000895CF93DF93EC0188818F
:10045000882329F08991E2DF88818823D9F7DF9109
:10046000CF9108952F923F924F925F926F927F9219
:100470008F929F92AF92BF92CF92DF92EF92FF92B4
:100480000F931F93CF93DF93CDB7DEB761970FB66E
:10049000F894DEBF0FBECDBFEE24FF2487018D8709
:1004A0006E877F876A01198A6624772423011301E6
:1004B00074C14989242F332720FF61C18889805363
:1004C0008A3008F46AC1E8898E2F992787FD9095B4
:1004D000883691055CF5853691050CF052C0833560
:1004E000910509F46CC084359105A4F48B32910513
:1004F00009F453C18C32910544F48032910509F41A
:100500004CC1839709F449C133C18D97029708F014
:100510002FC143C183369105B9F1843691050CF0A2
:1005200063C08835910509F48DC022C180379105DB
:1005300009F486C08137910584F48C369105E9F081
:100540008D3691052CF48936910509F44DC010C102
:100550008F36910509F470C00BC18537910509F4F8
:1005600074C08637910524F483379105A1F000C14A
:100570008837910509F466C0FBC0F989F460F98BEE
:100580000CC14FE3E42EAAC0F60182E090E0C80E51
:10059000D91EE080A0C0F60182E090E0C80ED91E0E
:1005A0000190F081E02D7F0144245524808188232F
:1005B00009F491C00894411C511C3196F7CFF60103
:1005C00082E090E0C80ED91E0190F081E02D7F01FD
:1005D0002F018491882329F00894411C511CF201B9
:1005E000F8CF4E185F0877C022FF0AC0F60184E0FA
:1005F00090E0C80ED91E20813181428153810CC008
:10060000F60182E090E0C80ED91E808191819C01A4
:10061000442737FD4095542F79018A0157FF2DC09B
:1006200099899260998B10950095F094E094E11C63
:10063000F11C011D111D21C038E0432E512C05C0B5
:10064000E8E7E88B90E1492E512C22FF0AC0F60121
:1006500084E090E0C80ED91E20813181428153810F
:100660000AC0F60182E090E0C80ED91E8081918117
:100670009C014427552779018A011E010894211CF9
:10068000311C4201AA24BB24C801B701A501940171
:10069000D8D0DC01CB01F10180838A3024F0F889C5
:1006A0008F0F815201C0805DF10181931F01C8014C
:1006B000B701A5019401C5D079018A012115310541
:1006C0004105510509F7F989F1FF05C08DE2A6DE64
:1006D0000894611C711C4889433611F48E2D49C061
:1006E00088898335D1F4640C751C0894410851083D
:1006F0009FEF49169FEF590609F43FC0F701089490
:10070000E11CF11C84918ADE089441085108EFEF46
:100710004E16EFEF5E0691F730C0F889F337C9F453
:10072000640C751C0894410851084FEF44164FEFB4
:10073000540619F1F7010894E11CF11C80816EDE6A
:100740000894410851088FEF48168FEF580691F72B
:1007500014C05E010894A11CB11C2A143B0469F06A
:10076000F10182911F015ADE0894611C711CF5CFC2
:10077000888954DE0894611C711C198A0EC0F8899E
:10078000F53231F441E0498B8AE0482E512C05C006
:10079000888944DE0894611C711C2E853F852F5F7B
:1007A0003F4F8D85813039F4EE85FF852E873F8759
:1007B0009491988B06C0EE85FF8580812E873F87B8
:1007C000888BF889FF2309F074CEC30161960FB6B8
:1007D000F894DEBF0FBECDBFDF91CF911F910F9177
:1007E000FF90EF90DF90CF90BF90AF909F908F9051
:1007F0007F906F905F904F903F902F900895CF9390
:10080000DF93CDB7DEB7E5E0F0E0EC0FFD1F81919F
:100810009191AF01BC0180E025DEDF91CF91089579
:10082000CF93DF93CDB7DEB7E5E0F0E0EC0FFD1F2F
:1008300081919191AF01BC0181E014DEDF91CF91F4
:100840000895A1E21A2EAA1BBB1BFD010DC0AA1F11
:10085000BB1FEE1FFF1FA217B307E407F50720F029
:10086000A21BB30BE40BF50B661F771F881F991FA4
:100870001A9469F760957095809590959B01AC01ED
:06088000BD01CF01089547
:100886000A0D53746172743A0A0D000A0D537461AD
:100896007274323A0A0D000A0D0A0D000A0D00257F
:0408A60075090000D0
:00000001FF
